:020000040800F2
:10000000001800200108000835050008390500081F
:1000100000000000000000000000000000000000E0
:10002000000000000000000000000000350500088E
:10003000000000000000000035050008350500083C
:1000400035050008350500083505000835050008A8
:100050003505000835050008350500083505000898
:100060003505000835050008350500083505000888
:100070003505000835050008350500083505000878
:100080003505000835050008350500083505000868
:100090003505000835050008350500083505000858
:1000A0003505000835050008350500083505000848
:1000B00035050008350500083505000899010008D8
:1000C000284B10B51A88284B12041B881A43274B5B
:1000D000198849084900885A254908801988023139
:1000E00089B21980198849084900885A214908802D
:1000F0001988023189B21980198849084900885A3B
:100100001D49088019881D48023189B21980198853
:1001100049084900895A1A4A11801A881949023235
:1001200092B21A801C880288944213D902881C88D3
:100130000832121B92B20A80028892B21A801249C7
:10014000124B0A881343124A1A40302353409BB281
:100150000B8010BD0F4804881A889442E6D3082308
:100160000B80ECE70C6000400A6000400460004037
:100170004C6000404E600040506000400260004013
:10018000526000401A600040005C00408080FFFF29
:10019000BF8FFFFF006000409449F8B50B88944C76
:1001A000002B3BD00A88934B9A4235D1002302257D
:1001B000914A1380914A1380914A1380914A138087
:1001C000914A1380914AD08FA843D087D08F013DA8
:1001D000A843D0878E481735C3878E4805808E4840
:1001E000343505808D480835058080258C486D01A3
:1001F000058080258B4805808548C38780208A4BF1
:1002000000062380894B18608023D08FDB000343D6
:10021000D387874A874B1A8000230B8023881BB221
:10022000002B00DBC3E02388834A764F13408022F3
:100230001343238023881B0500D49BE07F4D7F233D
:100240002A7811009943704B1980E9886A4B19800C
:1002500000216B4B19803B88FF318B4313433B805C
:1002600060231A4208D08022754B12051B88280093
:100270009B189847614B18802B78602259B200294F
:100280004DDA134014D16A78062A0FD16A88110A10
:1002900002291AD003291BD0012920D1694B12262B
:1002A000694A99B21180694A1B0C1380534B1E8016
:1002B0002288674B1343674A1A40C0239B0153406F
:1002C0009BB22380FFF7FCFE47E05E4B1233E6E76C
:1002D000D2B2012A0FD0002A03D0022A15D01E0064
:1002E000E4E7584B584A243399B21180574A1B0C03
:1002F00013800426DAE7534B534A283399B211800E
:10030000524A1B0C1380544ED0E74E4B4E4A7C335E
:1003100099B211804D4A1B0C1380504EC6E7134210
:1003200009D16B78052B06D13A886B88D2B21B02B3
:1003300013439BB23B8000212388494A1340494A1A
:1003400013439BB22380484B198023881A43474BA1
:100350001A40474B5A4092B222802D4BDB8F5B05EF
:1003600007D580222F4B1A800023294AD3872E4B92
:100370002380F8BD60213B880B40402BEDD13B88AA
:100380001342EAD1264A3B4B2C481B881188802215
:1003900012059B18C9B298472288324B13432D4A45
:1003A0001A40C0239B0153409BB22380D5E7802293
:1003B00023881342D1D023882F490B408021090282
:1003C0000B432380104B1B88934200D17AE7FF2018
:1003D0000C4B19888143C0D01988090A0A43114976
:1003E0000A801A8802401A80B7E7C0460E600040B3
:1003F000005C00403CA5000000600040026000403E
:10040000046000400660004008600040025C00405C
:10041000065C0040505C0040186000401C600040DA
:100420001E6000404C5C00402032000000E100E013
:100430000080FFFF585C00408F0F000054600040B8
:10044000106000407C0400080A6000400C6000401E
:100450008081FFFF8FBFFFFF2A0300001E03000003
:100460008F8EFFFF8080FFFF1A600040BFBFFFFF3D
:1004700030300000126000400F8FFFFF12010002B9
:10048000FF000008C016DC0502020102000109029B
:100490001200010100803209040000000000000089
:1004A000040309042A0349006E00660069006E0017
:1004B0006900740065004E00650073004C0069001F
:1004C0007600650073002E0063006F006D00000071
:1004D000000000000000000000000000000000001C
:1004E000000000000000000000000000000000000C
:1004F00000000000000000001E0349004E004C00F8
:10050000200052006500740072006F002D00500042
:1005100072006F0067000000000000000000000093
:1005200000000000000000000000000000000000CB
:1005300000000000FEE70000004801E02301ADDEFE
:10054000FEE7C04602B4714649084900095C49000B
:100550008E4402BC7047C046411D000000616561C9
:1005600062690001130000000536532D4D00060C92
:10057000074D09011901000003B471464908400004
:100580004900095E49008E4403BC7047411D0000CC
:100590000061656162690001130000000536532D9A
:1005A0004D00060C074D09011901000003B4714606
:1005B000490840004900095A49008E4403BC70476D
:1005C000411D0000006165616269000113000000C7
:1005D0000536532D4D00060C074D090119017047D2
:1005E0000A4B0B4A10B55A600A4A5A600122DC686D
:1005F0001442FCD11A6101220180D9681142FCD158
:100600002022DA6060321A6110BDC046002002402C
:1006100023016745AB89EFCDFF2370B53D4C2370B7
:10062000002363704378C588102B00D06FE0C37837
:1006300081888078384E01387269082800D964E0D2
:10064000FFF780FF0563632B3B3149515F008B1E31
:100650008E227D2B19D8314B7360314B736001238F
:10066000F2681A42FCD102233361802389021B0500
:10067000C918422371613361C046413BF2681A4098
:10068000FCD12023F360603333612270254BA2B28A
:10069000240CE8B25A819C8170BD58001018FFF7F5
:1006A0009FFF0022F1E78E22012BEED81804802351
:1006B0001B05C01840181C49F1E7042363707369D7
:1006C000A37073691B0AE37073691B0C2371736950
:1006D0001B0E6371E5E7022363701388A370138810
:1006E0001B0AE370DDE78E22012BCED880221B048B
:1006F00012059B185918022363700B88A3700B888E
:10070000EEE70A4A0A4BDA60CBE78B22BDE780238B
:100710002370BBE71A070020002002402301674531
:10072000AB89EFCD00600040FFFF00000400FA0538
:1007300000ED00E0000000000000000000000000EC
:1007400000000000000000000000000000000000A9
:100750000000000000000000000000000000000099
:100760000000000000000000000000000000000089
:100770000000000000000000000000000000000079
:10078000144B154A9BB21382144B9BB2538268469A
:100790001C300D4A0D4B0430043001681140C91A59
:1007A000FAD1074A074B043801681140C91AF2D13F
:1007B0007B460A33036004380133036008E0FEE738
:1007C0000000FFFF00000008FFFFFF0F0000000116
:1007D000002070471906000800600040DF0500088F
:1007E0000000000000000000000000000000000009
:1007F00000000000000000000000000000000000F9
:1008000009490A4A0A4B9B1A03DD043BC858D050D9
:10081000FBDC0849084A0020521A02DD043A8850DD
:10082000FCDC01F033FF000018500008000000203D
:1008300030040020300400202807002070B50F4C41
:100840002268537A55685A18D2B293420FD122685F
:100850000B48537ACB1853720378591AC9B20170F6
:100860000020814202D198230130D37070BD0678F8
:100870000130EE540133DBB2E7E7C0461407002035
:1008800018070020FF23F0B5B74C85B02370002374
:100890006370837905000093407801380E2801D9F0
:1008A00001F0B0FBFFF782FE0F00B1059B07A70820
:1008B0006B0AAE0B990B2D09D5091F0A680AE508CA
:1008C000F70809091B09A878AA888C2319281CD8BD
:1008D000FFF76CFE24002C0022011E02EA028903AD
:1008E0001804D404F004FC0404050C0515051E05C9
:1008F0002C0534053C0544051A001A001A00490568
:100900005E057505D202DE0200232370974B009826
:10091000A2B2240C5A819C8105B0F0BDB023944A48
:100920005B0351690B4353610023EEE7152A01D99C
:1009300000F05CFD1000FFF739FE160023002E00CA
:100940005905390044004F0059055C0069007300E7
:100950008000590559058D009A00A700B400C10018
:10096000CE00D800E2009023DB051A6881490A40D6
:100970001A608022D96852030A43DA600023C4E770
:1009800090230122DB05196891431960D9680A4355
:10099000DA600023B9E790230422DB05196891434C
:1009A0001960D9680A43DA600023AEE79023102269
:1009B000DB05196891431960D9680A43DA6000239E
:1009C000A3E790234022DB05196891431960D96899
:1009D0000A43DA60002398E79023DB051A6866492A
:1009E0000A401A608022D968D2040A43DA600023E0
:1009F0008BE79023DB051A6860490A401A60802261
:100A0000D96852010A43DA6000237EE704225C4B76
:100A1000196891431960D9680A43DA60002374E7C2
:100A20009023DB051A6857490A401A608022D9686A
:100A3000D2050A43DA60002367E79023DB051A68D2
:100A400051490A401A608022D968D2020A43DA600A
:100A500000235AE79023DB051A684C490A401A60C4
:100A60008022D96852000A43DA6000234DE79023C0
:100A7000DB051A6846490A401A608022D968D2000C
:100A80000A43DA60002340E79023DB051A684149F6
:100A90000A401A608022D968D2010A43DA60002332
:100AA00033E79023DB051A6833490A401A60802235
:100AB000D968D2040A43DA60002326E79023DB05D5
:100AC0001A6835490A401A608022D96852050A43DB
:100AD000DA60002319E70122294B19689143196054
:100AE000D9680A43DA6000230FE710222B4B1968FC
:100AF00091431960D9680A43DA60002305E790231F
:100B0000DB051A6822490A401A608022D968D2009F
:100B10000A43DA600023F8E6152A01D900F069FCDF
:100B20001000FFF743FD16003D0048006604530027
:100B30005E006900660474007F008900940066040A
:100B400066049F00AA00B500C000CB00D600E000FC
:100B5000EA009023DB051968064801401960DA684D
:100B60000240DA600023D0E6E40600200060004086
:100B700000100240FFFFEFFFFFFFFFFBFFEFFFFF53
:100B800000040048FFFFFFBFFFFFFBFFFFFEFFFF6A
:100B9000FFFBFFFFFFBFFFFFFFFFFFEF000C004861
:100BA00090230121DB051A688A431A60DA688A43B8
:100BB000DA600023A9E690230421DB051A688A4342
:100BC0001A60DA688A43DA6000239EE690231021D7
:100BD000DB051A688A431A60DA688A43DA60002300
:100BE00093E690234021DB051A688A431A60DA688D
:100BF0008A43DA60002388E69023DB051968CE4833
:100C000001401960DA680240DA6000237DE6902333
:100C1000DB051968C94801401960DA680240DA60EA
:100C2000002372E60421C64B1A688A431A60DA6808
:100C30008A43DA60002368E69023DB051968C1481F
:100C400001401960DA680240DA6000235DE6902313
:100C5000DB051968BC4801401960DA680240DA60B7
:100C6000002352E69023DB051968B848014019605B
:100C7000DA680240DA60002347E69023DB05196852
:100C8000B34801401960DA680240DA6000233CE6AC
:100C90009023DB051968AF4801401960DA6802400B
:100CA000DA60002331E69023DB051968A248014091
:100CB0001960DA680240DA60002326E69023DB053B
:100CC0001968A54801401960DA680240DA6000231B
:100CD0001BE601219A4B1A688A431A60DA688A4334
:100CE000DA60002311E610219C4B1A688A431A60CF
:100CF000DA688A43DA60002307E69023DB05196887
:100D0000934801401960DA680240DA600023FCE58C
:100D1000152A00D970E31000FFF748FC16001F00E9
:100D200027006E032F0037003F006E03480051007C
:100D3000580061006E036E036A0073007C0085003A
:100D40008E0097009E00A50090228023D205116896
:100D50005B030B4313600023D7E590220123D205E8
:100D600011680B4313600023CFE590220423D205C2
:100D700011680B4313600023C7E590221023D205AE
:100D800011680B4313600023BFE590224023D20576
:100D900011680B4313600023B7E590228023D2052E
:100DA0001168DB040B4313600023AEE5902280231F
:100DB000D20511685B010B4313600023A5E50423F2
:100DC0005F4A11680B43136000239EE59022802345
:100DD000D2051168DB050B431360002395E59022D3
:100DE0008023D2051168DB020B43136000238CE5DE
:100DF00090228023D20511685B000B43136000230F
:100E000083E590228023D2051168DB000B43136039
:100E100000237AE590228023D2051168DB010B4381
:100E20001360002371E590228023D2051168DB0452
:100E30000B431360002368E590228023D2051168DC
:100E40005B050B43136000235FE501233C4A1168F7
:100E50000B431360002358E51023404A11680B43ED
:100E60001360002351E590228023D2051168DB0036
:100E70000B431360002348E58D23082A00D044E586
:100E800090224023D20551680B43536000233CE578
:100E90008D23082A00D038E590224021D2055368DE
:100EA0008B435360002330E5152A00D9A7E21000D8
:100EB000FFF77CFB16001D002300A50229002F0070
:100EC0003500A5023C0056005B006200A502A502A9
:100ED00069006F0075007B00820089008E0093001E
:100EE00080229023D200DB059A6200230DE5902337
:100EF0000122DB059A62002307E590230222DB052D
:100F00009A62002301E590230422DB059A62002304
:100F1000FBE490230822DB059A620023F5E480229B
:100F200090239201DB059A620023EEE49023402295
:100F3000DB059A620023E8E4FFFFFFFBFFEFFFFF02
:100F400000040048FFFFFFBFFFFFFBFFFFFEFFFFA6
:100F5000FFFBFFFFFFBFFFFFFFFFFFEF000C00489D
:100F60000222CF4B9A620023CFE480229023120208
:100F7000DB059A620023C8E4802290239200DB05FF
:100F80009A620023C1E490231022DB059A620023B9
:100F9000BBE490232022DB059A620023B5E4902372
:100FA0008022DB059A620023AFE480229023920125
:100FB000DB059A620023A8E480229023D201DB059E
:100FC0009A620023A1E40122B54B9A6200239CE4BB
:100FD0000422B44B9A62002397E490232022DB057D
:100FE0009A62002391E4152A00D90BE21000FFF762
:100FF000DDFA16001D002300090229002F0035002C
:1010000009023C00420047004E0009020902550057
:101010005B00610067006E0076007C008200802229
:101020009023D200DB059A6100236EE49023012215
:10103000DB059A61002368E490230222DB059A61B4
:10104000002362E490230422DB059A6100235CE420
:1010500090230822DB059A61002356E48022902326
:101060009201DB059A6100234FE490234022DB05C7
:101070009A61002349E40222894B9A61002344E4E7
:10108000802290231202DB059A6100233DE4802236
:1010900090239200DB059A61002336E4902310220E
:1010A000DB059A61002330E490232022DB059A615E
:1010B00000232AE490238022DB059A61002324E4A4
:1010C000802290239201DB059A6100231DE4802297
:1010D0009023D201DB059A610023FFF716FC012261
:1010E0006F4B9A610023FFF710FC04226D4B9A614D
:1010F0000023FFF70AFC90232022DB059A610023DE
:10110000FFF703FC02236370152A00D9B1E0100039
:10111000FFF718FA0B151EAF273039AF434C545D5B
:10112000AFAF677079828C969EA690238022DB05F4
:101130001B69D200134063800023FFF7E6FB902376
:101140000122DB051B69134063800023FFF7DDFBF1
:1011500090230222DB051B69134063800023FFF705
:10116000D4FB90230422DB051B691340638000231A
:10117000FFF7CBFB90230822DB051B69134063803C
:101180000023FFF7C2FB90238022DB051B6992013D
:10119000134063800023FFF7B8FB90234022DB0558
:1011A0001B69134063800023FFF7AFFB02223C4B17
:1011B0001B69134063800023FFF7A7FB9023DB0527
:1011C0001B69DB0BDB0363800023FFF79EFB90238F
:1011D0008022DB051B699200134063800023FFF728
:1011E00094FB90231022DB051B69134063800023CE
:1011F000FFF78BFB90232022DB051B6913406380E4
:101200000023FFF782FB90238022DB051B6913403C
:1012100063800023FFF779FB90238022DB051B69A5
:101220009201134063800023FFF76FFB902380221D
:10123000DB051B69D201134063800023FFF765FBC8
:101240000122174B1B69134063800023FFF75DFBEE
:101250000422144B1B69134063800023FFF755FBE6
:1012600090232022DB051B69134063800023FFF7D6
:101270004CFB002363708D33FFF747FB80230A4A42
:10128000DB0251690B435361054B08491A680A4058
:101290001A60D968064A0A43DA600023FFF735FB73
:1012A00000040048000C004800100240FFFFAAAAFA
:1012B00000005555EF4BF0491A680A401A60D9688A
:1012C000EE4A0A43DA600023FFF71FFBE94AEA49C6
:1012D00013680B4013600023FFF717FBE54AE74B49
:1012E00011680B4313600023FFF70FFBE149120263
:1012F0004B69DBB21A434A610023FFF706FBDD4B63
:101300001B691B0AA370012363700023FFF7FDFA1A
:101310008023DB4A1B0351690B435361D94ADA4BE3
:1013200011680B4313600023FFF7EFFAD54AD64B41
:10133000D1680B43D3600023FFF7E7FAD14AD349C2
:1013400013680B4013600023FFF7DFFACD4ACE4B42
:1013500011680B4313600023FFF7D7FAC94B5A619A
:101360000023FFF7D2FAC023C54ADB0251690B43C1
:101370005361C04AC64B11680B4313609022A023EF
:10138000D20511685B030B4313600023FFF7BDFA1E
:10139000B84ABF4BD1680B43D3609023A021DB0533
:1013A000D86849030143D9601168BA480140116007
:1013B0001A68B9490A401A600023FFF7A6FAFF2508
:1013C000AC48930041692B40B44DD20029400B43F7
:1013D00043619021C020C905C0004B690240B0485C
:1013E00003401A434A610023FFF78FFA8D23FFF76A
:1013F0008CFA8D23FFF789FA8D23FFF786FA8D2368
:10140000FFF783FA8D23FFF780FAAA88AD78032DC2
:1014100000D10BE155D8012D63D05ED901F08CF8D5
:1014200090220121D20513680B43136010239161B0
:1014300011680B43136004234021936113680B432D
:101440001360082393619161802311685B010B4352
:10145000136080238A48DB024169874E0B4385492C
:1014600043610B6833400B60CD68844B1D43CD60F6
:101470000C6834400C60CC682343CB608023446903
:101480001B0323437F4C436125687F4B2B43236021
:1014900000236361C0244569E4022C4344610C6865
:1014A0007B4820430860A02014684003204310605C
:1014B00048697A4C2040486151697948014051613E
:1014C00051E0052D52D000D211E1072D00D191E05D
:1014D000802D00D130E1962345E001F02DF8002366
:1014E00041E001F029F89023DB051A682A431A60CD
:1014F00080229D61196852030A431A6080220421E8
:10150000D2009A621A685C4D0A431A6002229A61FC
:1015100018680E3202431A604022996119680A4322
:101520001A6008229A618023554ADB0251690B43F5
:101530005361504B196829401960DC684F490C43CE
:10154000DC60186828401860D8680143D96080239F
:1015500051691B030B4353614A4A4B4B11680B43C0
:101560001360002353614F4CFFF7CFF900F0E4FF05
:1015700090220121D20513683F4E0B4313601023C4
:10158000916111680B431360042340219361136838
:101590000B431360082393618023916211685B0100
:1015A0000B43136080233649DB02486903434B61D8
:1015B000304B186830401860DD6830480543DD6006
:1015C0001C6834401C60DC682043D8608023486974
:1015D0001B0303434B612B492B4B086803430B60F0
:1015E00000234B6180211068C901014311608021F3
:1015F0009162B8E700F0A0FF90220121D2051368A4
:1016000040200B4313601023916111680B4313605A
:1016100004239361116801431160082191611168ED
:101620000B4313600223936190610DE7D2B2022A4B
:101630003ED00023032A96D09723012A93D18023FA
:101640000F491B03486903434B610E490B689343E1
:101650000B60CB681343CB604B6813434B608A61CC
:101660000B681A4300230A600F4A13700F4A116077
:1016700079E7C04600040048FFFFAAAA00005555BC
:10168000001002400008004855555555AAAAAAAABC
:1016900050550000AFAAFFFFFFFFEBFF03FF000064
:1016A000FFF90000E4060020F0060020EC06002010
:1016B000B023B74A5B03516940200B435361902329
:1016C000DB051A68B3490A401A608022D9685201C2
:1016D0001143D960596801435960986119680A43F8
:1016E00008211A60AC4A1170AC4A1360F7E6D2B216
:1016F0009823012A00D036E79022A94BD2051A6020
:1017000006220A21A74B1A70A74BA84A1360A84AC1
:101710001170A84A01311360A74A1170A74A1360DB
:101720000C22A74B1A70B023994A5B0351690B43F3
:10173000536100F025FED2E690230125402180264A
:10174000DB05657099621A68760132431A60C046FB
:1017500090481C691A680C4002401A60DA6802401E
:10176000DA60F022002C37D11A6802401A60DA6879
:101770001643DE601A6994461A690192C0461A69D6
:101780000292C046C0461A690392C046C046C0468F
:101790001F69C046C046C046C0461E691A6802405E
:1017A0001A60DA681040D860634622000B4213D1F9
:1017B000019B2A000B420FD1029B02320B420BD13C
:1017C0000B0003990332194206D104321F4203D1A0
:1017D00005321E4200D1D1327A4B9A707FE6E97809
:1017E000A888AD780D2D00D195E023D8062D56D0D0
:1017F0000FD8022D5AD005D8002D4BD0012D52D034
:10180000A02549E0042D74D0052DF9D101F042FE48
:1018100047E0092D76D007D8072D00D181E0082DAB
:10182000EED101F03DFF3CE00B2D77D06DD901F0FA
:10183000B9FE36E0222D3CD011D8102D74D006D838
:101840000E2D65D00F2DDBD101F08CFF29E0202D6E
:1018500052D054D8112DD3D101F0E8FE21E0822DD1
:1018600000D190E009D8802D61D0812DC8D101230D
:10187000637001F0C9FFA07013E0852D00D1ADE0C9
:10188000862D00D1AFE0842DBAD10123637001F021
:1018900029FEF0E700F048FD2570FFF737F802F069
:1018A000A1F80025F8E701F039FEFAE701F000FDA4
:1018B000F7E7454B902258610223D20593623A4BD9
:1018C000424D1E68090235431D605D6900B2EDB2EC
:1018D00029435961002801DA01219162C046C046BE
:1018E00001219161491891611A6839490A401A60C9
:1018F000D7E702F00DFAD4E7364B1870D1E7364B34
:101900001880CEE702F04CF8CBE701F05BFFC8E7A8
:1019100002F01EF8C5E701F0E9FFC2E701F0E2FEC0
:10192000BFE701F0BBFFBCE701F08EFFB9E7012183
:1019300090236170DB051D68164E35401D60DA6826
:1019400002253240DA608022D2009A6299619D615C
:101950001D4D6861C046C04600B29A61002800DA99
:101960009962C046C046C046C046C046C0469022A6
:1019700080210D4BD205C9001B69916201211B0A10
:101980009161A3708DE70123637001F0EFFD72E7B1
:1019900000100240FFEFFFFFF0060020EC060020E1
:1019A000040700200807002000040048FC0600206F
:1019B000000700200C07002010070020F40600207C
:1019C000F8060020E40600200008004800005555F5
:1019D000FFFFAAAA880400203404002001236370BA
:1019E000C74B1B78CDE702236370C64B1B88A370DF
:1019F0001B0AE37055E7A878E978AB88AA22062885
:101A00001AD8FEF79FFD042B1C2327332100FF2546
:101A1000BD489A0041692A40BC4DDB0029400A4379
:101A200042619021C020C905C0004A690340B848FE
:101A3000024013434B6100222270FEF767FF002231
:101A4000180001F091FBF6E70122F9E7180001F018
:101A500007FCF0E7180001F0DBFBECE701220021B6
:101A60006270180001F0B0FBA070E4E70121617022
:101A7000F7E7AA78002A07D00023012A01D1FEF750
:101A800044FFAF23FEF741FF01236370A933A37026
:101A90001300FEF73AFFAA78002A07D00023012A94
:101AA00001D1FEF732FFB023FEF72FFF0123637051
:101AB000A933A3701300FEF728FFAA78002A07D0E5
:101AC0000023012A01D1FEF720FFB123FEF71DFFFD
:101AD00001236370A933A3701300FEF716FFAA78E1
:101AE000002A07D00023012A01D1FEF70EFFB223FE
:101AF000FEF70BFF01236370A933A3701300FEF7F9
:101B000004FFEA78A988AD78112D00D19AE007D8B2
:101B1000012D6BD0002D0FD0022D7CD08225BBE68D
:101B2000212D00D184E0222D00D187E0122DF5D1A6
:101B300002231020637088E001263100754D764F36
:101B40002A783B68914099625A6810208A435A600B
:101B500001F094FC31002B783A6899400B00FA2789
:101B60000425916151687F000B4353600196380052
:101B700001F084FC674A01991278674E91403368FE
:101B8000380099625A68013D8A435A6001F076FC38
:101B9000604B01991B78326899400B009161516844
:101BA000ADB20B435360002DE1D1FA270435380064
:101BB00001F064FC0121574A574E12783368914076
:101BC00099625A6838008A435A6001F057FC012133
:101BD000504B32681B78013D99400B009161516870
:101BE000ADB20B435360002DE1D155E62900494EBB
:101BF000494F32783B68914099625A6810208A4375
:101C00005A6001F03BFC32783B6895409D615A6810
:101C100015435D6045E601233E4A637012783F49F3
:101C200093403D4A9BB21268002002F089F822E6F8
:101C300001230020637001F071FB1CE601231020DA
:101C40006370F8E702230020637001F0C1FB60803D
:101C500027E6AB78AA88042B1DD007D8022B1FD00B
:101C600024D8012B12D08723FEF74FFE072B26D056
:101C700003D8052BF7D12A4B16E0082B24D0802B54
:101C8000F1D100F07DFB0023FEF73FFE254A1278DC
:101C9000A2706370F7E7244B1B78A3700123F8E769
:101CA000204B1A708322204B1A70ECE71D4B1E4DFF
:101CB0001A7083232B7000F0D3FB2B78EDE71B4BBE
:101CC0001A70120A5A70DEE7184B1A78A2705A7806
:101CD000E2709A782271DA7862711A79A2715B796E
:101CE000E3710623D5E7A878AA8801388A23032858
:101CF00001D9FEF70AFEFEF725FC1B30333AC04639
:101D000088040020340400200004004803FF000081
:101D1000FFF90000F0060020EC060020040002009D
:101D2000D1040020B0040020D2040020B10400201F
:101D3000024885460248001C0047C0467812002031
:101D4000C5CAFF1F060005000800070019C9FF1FCC
:101D5000EFBEADDE0023FEF7D8FDBE4B1A60F9E7FB
:101D6000BC4B18680004104301F0E4FFF2E7FEF7F3
:101D700007FD0300FEF7C9FD8823FEF7C6FDAA781C
:101D80001300303B2F2B1CD8E878032816D8FEF719
:101D9000D9FB18021113B04B512A00D183E029D886
:101DA000312A5BD00FD8002A39D0302A4FD0B42343
:101DB000FEF7ABFDA94BEFE7A94BEDE7B523FEF727
:101DC000A4FDA84BE8E7332A56D04ED3502AEED1D3
:101DD00000222270063262701A7AA270DA78E270FB
:101DE0005A7A22719A7A62719A78A2715B7CE37155
:101DF000FEF78CFD7F2A00D989E0702A63D2602A21
:101E00003FD0612A47D0522AD1D100221B882270AC
:101E1000A37002321B0A6270E370FEF777FDFF23A6
:101E2000914953540132102AFBD18B4A8D49D3700A
:101E300093708B4ACB70D370937001228B7087495B
:101E4000CB708B70894B1A700023FEF75EFDAA8859
:101E5000110AD9721A730023FEF757FDAA88110AD6
:101E600059739A730023FEF750FDAA88110AD9739B
:101E70001A740023FEF749FDAA885A740023FEF75E
:101E800044FD0023237001336370AB88764AD35C32
:101E9000A370FEF73BFD0023237001336370744B86
:101EA0001B68DB78F4E70022227006326270DA7A6F
:101EB000A2701A7BE2705A7B22719A7B6271DA7B84
:101EC000A2711B7C93E7674B69495C682B787F2B79
:101ED00000D99AE06846674B007818700B68D8788C
:101EE00000280DD000230093982805D195E0002309
:101EF0000093D02800D190E010205C4B187003E0D4
:101F00005D4803609020D870FF23009385E0072090
:101F1000104003281AD8FEF715FB1C021E174E4B63
:101F2000802A01D2FEF7F2FC872A16D97032D2B28B
:101F3000072A01D9FEF7EAFC00222270EA789A7299
:101F4000AA881A80FEF7E2FC454BE9E7B523FEF7C5
:101F5000DCFC444BE4E7414BE2E7A888E978C6B2F1
:101F60008D19BE22102D00DD66E50432002900D156
:101F700062E5DD78033AFF2D00D05DE59D78013202
:101F8000FF2D00D058E50022374DD7B2B9421CD8FA
:101F90004F01013F1F727701BC460022374F000AF4
:101FA00067449870DA705A729A721A80DA721A73E9
:101FB0005A739A73DA731A745A745F60AD19A8541D
:101FC0000132D3B29942FAD835E50132B718013F50
:101FD000EF5DFF2FD9D0C1222EE5AB78002B04D0C6
:101FE000402B08D0D223FEF790FC2370AA881F4B09
:101FF0001A70FEF78BFC00232370013363701B4BB8
:102000001B7845E78023FEF780FC0B68D878D8283A
:1020100000D06CE780205C68D8700B680021597292
:10202000DB78902B01D0FEF771FC712A01D0FEF70E
:102030006DFC114BA9881A68526811701A685168B2
:10204000AA88120A4A701A68537A02335372FEF74A
:102050005DFCC046300400204C04002060040020D9
:102060007404002038040020D304002090040020D1
:102070008C0400201807002014070020E40400202E
:10208000F0B5404B8BB0089119783F4B09921B7803
:10209000019002933D4B019D1C683D4B3D481A78D1
:1020A00001231E0096403C4AA662102D5ED1127894
:1020B00000689340836201200200364B05901F6840
:1020C000354B1B789A4003920200344B1B680693F1
:1020D000334B1B789A4093B202000793314B1B6835
:1020E0009C46314B1B789A40002304921A000198B9
:1020F000202806D1029D05981D4105423ED0039837
:10210000B861089820280FD1002B01D11E488354B4
:10211000069805690798054206D01B48855C059816
:10212000984005431848855409980139C9B20028D8
:1021300002D0002900D1A6616046049D0133DBB2C4
:1021400085618562082B05D101320F4BD2B29B5CB1
:10215000029300230029CAD10E4B1A680E4B19783E
:1021600001238B409362A6620BB0F0BD019D112D3F
:10217000A1D112780068934083619CE70398B8620C
:10218000BFE7C046D1040020B10400200C070020A6
:1021900010070020FC060020000700200407002094
:1021A00008070020F4060020F8060020F7B51F4BB2
:1021B0001F491A781F4B10282ED101241E780D6854
:1021C000B440AC62012635000C6831001B780196E2
:1021D0009D40194B1B680093184B1B7899400023B6
:1021E0008C46190020280DD1154E019F765C1E41AA
:1021F0003E4219D0A5610133DBB2082B02D1002386
:102200000131C9B26646009F013AD2B2BE61BE62D8
:10221000002AE7D1A562F7BD1128D3D101241E7889
:102220000D68B440AC61CDE7A562E4E7D1040020BD
:102230000C07002010070020F4060020F8060020FC
:10224000B1040020F7B50D00042701924C7A00027A
:1022500003B2A6B200932B7AB34202D26C72002072
:10226000FEBD00986B682043195D80B2019B9847C2
:102270006B681A5D094B824205D01A683A431A60AE
:1022800002229A61E7E71A680134BA431A60DA68F1
:1022900001363A43DA60E4B2B6B2DCE70004004843
:1022A000F7B50D001600FF27000203B24C7A019328
:1022B0002A7AE3B2A24202D26B720020FEBD200055
:1022C0006A683840D15C019B0134184380B2B04742
:1022D000A4B2EDE7022907D10F4B104A984218D05B
:1022E000904209D1180007E0032906D10A4B0B4997
:1022F0000B4A98420BD1080070470429FCD1064BC9
:10230000064A984205D006499042F4D0054A8842D0
:10231000E6D11000F0E7C046380400204C0400204D
:102320006004002074040020104B114A10B558615D
:102330001068104B09020343136053690E4CDBB263
:102340001943902351618021DB0518684901084336
:10235000186040209862186820401860D8680143CF
:10236000D960136805490B40136010BD0008004890
:102370000004004800005555FFEFFFFFFFFFAAAA29
:10238000F0B52C4B85B019682B4B2C481B78007886
:102390000193012302901E0018001F00019A029C65
:1023A0009640A040264D274A2D781268AF408E6295
:1023B0008446906224489D400068876204680394C4
:1023C0001C00AC402500039C254305604568019C2A
:1023D000BD4345609C401D00A54008681C00284383
:1023E00008604868B04348601068029999408C4082
:1023F00021000143604611605168814313485160D8
:102400000078134A98408340126812481168994333
:102410001160D1680B43D36080220F4B1A700023E8
:1024200019000E4A13701A1801331170202BFAD1BB
:1024300005B0F0BD0C0700201007002000070020A9
:10244000F8060020FC060020F40600200807002003
:1024500004070020B1040020D2040020D104002091
:1024600010B5334B1B78082B5DD016D8314C032B9D
:1024700044D007D8012B2DD0022B31D0EE222D4B8A
:102480001A7023E0062B44D049D8042BF6D18123BF
:10249000012223702021112027E00F2B34D008D8EF
:1024A000244C0D2B25D00E2BE8D181230022237044
:1024B00027E0802B08D01F4CFF2B08D0102BDDD13C
:1024C00081230022237027E0FFF75AFF10BDF0237D
:1024D0002370FBE7812320202370FFF767FE06E0CF
:1024E00081230122002123702020FFF7C9FD8223D0
:1024F000EEE78123002223701100F5E781230122FA
:10250000237020211020F0E781230A4C0022237041
:10251000C0E781230122237020210800E5E7812301
:1025200010202370D9E78123024C11202370D4E7B7
:10253000B0040020D2040020BC234749DB038A6A90
:10254000F0B513438B628B6A444A012413408B62BB
:1025500090238022DB051868D20102431A60802292
:102560009A61B0224869520302434A611A683C48A2
:102570003C4F02401A608022D86852030243042074
:10258000DA601A68A2431A60DA682243DA601A68CD
:1025900082431A60DA680243DA6010221D689543AC
:1025A0001D60DD682A43DA6040221D6895431D6086
:1025B000DD682A43DA601A682B4D2A401A608022AF
:1025C000DD68D2042A43DA601A68284D2A401A606E
:1025D0008022DD68D2052A43DA601A68244D2A4039
:1025E00080251A60DA68ED022A43DA60214A16680B
:1025F000A6431660D6683443D4601E683E401E6011
:10260000DC683C40DC6080234C691B0323434B6146
:10261000194B1A4C1E681A4F26431E601E683E4016
:102620001E60DE683443DC604B691D434D611368F6
:10263000144D2B401360D468134B1C43D4601168B5
:1026400029401160D1680B43D36013688343136042
:10265000D3681843D060F0BD00100240FFFFA1FF17
:10266000FFFFEFFFFFEFFFFFFFFFFFFBFFFFFFBFDE
:10267000FFFFFBFF00040048000800485555555572
:10268000AAAAAAAAFFFFAAAA000055559022D34BD6
:1026900012031968F0B50A431A60802289B09202C9
:1026A00019681142FCD0012259680A435A608022FD
:1026B000596852020A435A608022596852030A43F9
:1026C0005A608022196852040A431A6080229204D8
:1026D00019681142FCD01121C14AC24C11605A68DC
:1026E0000E398A43110002220A435A608022196B74
:1026F0000A431A638022D96912040A43DA61BA4B89
:10270000E381BC231B689847B84B6382B84B238294
:1027100062B6FFF711FFF022B64B1A70B64E2023B7
:10272000327811009943D2292ED1B449B448C978DE
:10273000C3780224FF2904D1FF3B1C00631E9C4187
:10274000E4B2B04BDB78FF2B00D00324AE4BDB7838
:10275000FF2B00D00424AD4BAD4F1C703860D22A43
:1027600012D10023012505E02100FFF7B3FD01236D
:102770000135EDB2A542F7D3002B00D0386080229E
:102780003B68DA70D02333703378F22B05D1002206
:10279000023B33709E4B1B68DA703578D02D01D028
:1027A00000F07EFC9A4E3068C378802B01D000F098
:1027B00077FC964B1978FFF78DFD002330600400FD
:1027C000C57006884372C07AF5B21038152801D951
:1027D00000F064FCFDF7EAFE52008A00D200D60049
:1027E00062046204620462046204620462046204B9
:1027F00062046204620462041600250036003B0095
:1028000041004B00E17BC4230F2901D900F047FCB4
:1028100009013143237AA278C9B2606801F00EFA47
:102820000EE0E17B3C230A009A438833002A01D062
:1028300000F035FC237AA2782943606801F034FA6D
:10284000607292E0237AA278E17B2943E5E7E17B9D
:102850003F230A009A438533E8E7227AE17BA37895
:10286000009200222943606801F0AAF9E8E7E17BC1
:10287000227AA378294300920122F4E7E37B1E2BFE
:102880000BD1C020B6092233F1B200029D4300F003
:102890000FFD237AA2788021D7E71C2B0FD1A0202F
:1028A0008121C00100F004FD8020F609F1B2000290
:1028B00000F0FEFCA0200021C00100F0F9FC802106
:1028C000E27B49421F2A05D00D43EDB2237AA2785C
:1028D0002900A2E77022A02095430D432188C00162
:1028E0000909C9B2EDB200F0E3FCEFE7E37BFE2B90
:1028F0003BD17609F1B2474800F010FE1F21464B4C
:102900000D405A692D02D2B2154380219022C90090
:10291000D205A0786768267A5D6191610121FF2563
:102920009162033191625A692D022A4002435A6131
:10293000C0463A4900228C46C046614609690130CA
:10294000090AB9545969C0B2294001320143D2B2CF
:1029500059619642F0D290230421DB0599618021D0
:10296000C9009962012199616272294B1B6819881B
:102970009A7A52181A80D822DA7091E3237AA278D0
:10298000602162E7E37B002B20D18033F6091D43F1
:10299000F3B20293FF20029B20499B004A69034047
:1029A0001F48024013434B61C0209021029BC90580
:1029B000C000DB004A6903401A48024013434B61E0
:1029C000227AA3782900009200224CE7012BE1D162
:1029D0004021B604B60E31430291DBE700100240FD
:1029E00000200240006000403CA5FFFF3D080008B9
:1029F00085080008D2040020900400204C04002028
:102A00003804002060040020740400201107002016
:102A10008C040020FF3F000000080048000400482C
:102A200003FF0000FFF90000E37B002B06D130001C
:102A30008038C0B2D14A2100FFF704FCE37B012BB0
:102A400006D130008038C0B2CD4A2100FFF728FC03
:102A5000E37B032B06D130008038C0B2C94A210085
:102A6000FFF71EFCE37B042B06D130008038C0B298
:102A7000C54A2100FFF7E6FBE37B0A2B06D13000B5
:102A80008038C0B2C14A2100FFF70AFCE37BFD2B6E
:102A900015D13F20238830409B0904936B46802644
:102AA0001B7C06430693677ABBB2039333021BB2C7
:102AB0000793237A039A934200D3AAE06772E37BD9
:102AC0001E2B11D13F2030408026238806439B09CE
:102AD000DBB20593657A33021BB2AFB20693237A59
:102AE000BB4200D3DDE06572E37B0C2B17D11F20C6
:102AF000304080260643C0202588A5216D09EDB20F
:102B0000C00100F0D5FB2900A14800F0D1FB677A95
:102B100035023D43237ABB4200D311E16772E37B68
:102B20001C2B3BD1A02023888121DB09DBB2C00113
:102B3000049300F0BDFB80200499000200F0B8FB74
:102B4000A0205421C00100F0B3FB677AAA21BBB2D8
:102B50009048039300F0ACFB55218F4800F0A8FB90
:102B600020218C4800F0A4FB802333431B021BB2BE
:102B70000693237A039A934200D31FE18020902189
:102B80000002677200F094FB80200021000200F038
:102B90008FFB8020F021000200F08AFBE37B1F2BDB
:102BA00030D1A0202188C0010909C9B200F080FB02
:102BB000AA217848657A00F07BFB5521764800F021
:102BC00077FB7448202100F073FB702380209E4324
:102BD0004042304340B20302AFB20493237ABB4277
:102BE00000D333E1802090210002657200F060FB89
:102BF00080200021000200F05BFB8020F021000219
:102C000000F056FBF4232288E370A37A9B182380FC
:102C100066E20021614800F04BFBAA21604800F009
:102C2000E1FE55215F4800F0DDFEA0215C4800F088
:102C3000D9FE6B46187C5C4B0699C01880B200F038
:102C400037FB079D63683D43ADB2D95D280000F0B6
:102C5000C9FEC046280000F0D7FD0590280000F00E
:102C6000D3FD059B8342F4D163680599DA5D4F4B30
:102C70008A420FD1039A1968013292B20392042258
:102C800091431960D96801370A43DA600222FFB222
:102C90009A620EE7042219680A431A6002229A61B6
:102CA00007E7C0200121000200F002FBAA214048F2
:102CB00000F0FEFAC0200021000200F0F9FA5521D0
:102CC0003C4800F0F5FAC0200121000200F0F0FAC3
:102CD000A021374800F0ECFAC0200599000200F06E
:102CE000E7FA069B2B439BB2039363680398595DF5
:102CF00000F0DEFAC046039800F086FD04900398C9
:102D000000F082FD049B8342F4D1636804995A5D0C
:102D1000264B8A420DD1042219680135914319606E
:102D2000D96801370A43DA600222EDB2BFB29A6273
:102D3000D5E6042219680A431A6002229A61CEE697
:102D4000AA211D4800F0B4FA55211A4800F0B0FA43
:102D5000A021194800F0ACFA63682800D95D00F0A2
:102D6000A7FAC046280000F04FFD0390280000F0AD
:102D70004BFD039B8342F4D1CCE6C046A139000849
:102D800051390008ED3800089D380008493800081E
:102D9000FFFF0000AA8A00005585000069FD0000C1
:102DA00055550000AA2A000069FDFFFF00040048F5
:102DB00055950000AAAA000055D50000A020542176
:102DC000C00100F075FA069DA0213D43ADB2280078
:102DD00000F06EFA63682800D95D00F069FAC04619
:102DE000280000F011FD0590280000F00DFD059B66
:102DF0008342F4D16368059ADB5DC04D93420FD1E5
:102E0000039B2A6801339BB2039304239A432A60ED
:102E1000EA6801371343EB600223FFB2AB62A8E616
:102E2000A0208121C00100F043FA80200499000213
:102E300000F03EFAA0205421C00100F039FA04232A
:102E40002A6813432B600223AB6192E6049EA02103
:102E50002E43B6B2300000F02BFA63683000595DA3
:102E600000F026FAC046300000F0CEFC039030009F
:102E700000F0CAFC039B8342F4D1636803995A5D56
:102E80009E4B8A420DD104211A6801358A431A608B
:102E9000DA6801370A43DA600222EDB2BFB29A6201
:102EA0009CE604211A680A431A6002229A6195E698
:102EB000E37B002B04D1924A21003000FFF7F0F9A8
:102EC000E37B012B04D18F4A21003000FFF7E8F9A2
:102ED000E37B022B04D18C4A21003000FFF7E0F99C
:102EE000E37B042B04D1894A21003000FFF7D8F995
:102EF000E37B0A2B04D1864A21003000FFF7D0F98A
:102F0000E37B0B2B04D1834A21003000FFF7C8F983
:102F1000E37BFE2B00D075E621887F484909C9B2C2
:102F200000F0FCFAAA217D48657A00F0B3FA552139
:102F30007B4800F0AFFA7948202100F0ABFA1F205F
:102F400030400302AFB20493237ABB420DD26572C4
:102F50009021002000F09EFA0021080000F09AFA6B
:102F6000F021002000F096FA4CE6049EA0212E43AA
:102F7000300000F08FFA63683000595D00F08AFA83
:102F8000C046300000F0AEFA0390300000F0AAFA1C
:102F9000039B8342F4D1636803995A5D574B8A427D
:102FA0000DD104211A6801358A431A60DA680137A5
:102FB0000A43DA600222EDB2BFB29A62C4E704218A
:102FC0001A680A431A6002229A61BDE73000603035
:102FD000544A2100C0B2FFF763F913E6E37B042BE8
:102FE00006D130008038C0B24F4A2100FFF758F9AF
:102FF000E37B052B04D14C4A21003000FFF750F948
:10300000E37B062B06D130008038C0B2474A21004E
:10301000FFF746F9E37B072B04D1444A2100300037
:10302000FFF73EF9E37B002B1CD1FF2580331E43C5
:1030300023883248DB09DBB29A0041692A403C4DC3
:10304000DB0029400A4342619021C020C905C0002D
:103050004A6903403748024013434B613000210066
:1030600000F0E4FCE37B012B00D0CBE52388234A6E
:103070002F4851699B049B0E01409B000B439021FC
:103080005361C9054B692B4A30001A4080239B00CD
:1030900013434B61210000F0C9FCB3E5C323E37087
:1030A000254B1D78F02D1BD1244E3468E378982BE6
:1030B00016D1234B20001978FFF70CF9002330605C
:1030C000C370E07AE57010382678042806D8FDF73A
:1030D00053FAABFCEFFE7DFF85FF99FDC323E37040
:1030E000184B1B78F02B01D1FFF718FB832B01D075
:1030F000FFF714FBFFF7B4F9FFF710FB00040048DB
:10310000C537000865370008E5360008A136000815
:103110002D360008A5350008FF3F0000AA0A000070
:1031200055050000B1320008613200081132000874
:1031300003FF0000FFF90000900400208C04002031
:1031400011070020D2040020002302000002002A00
:1031500004D1002B01D0802318437047DB43511E5C
:10316000DBB20A40F3E70000134B10B55861134B74
:1031700013481C680902204318605869C0B2014313
:10318000596190210820C9058862002A01D10132C5
:103190008A62C046C046C046C046C046C046C04619
:1031A000C04690220821D2059161073991611A68C1
:1031B00004490A401A6010BD000800480004004895
:1031C00000005555FFFFAAAA0F4B58619023DB055D
:1031D000002901D101229A6204229A62C046C046A7
:1031E000C046C046C046C046C046C046C046C046AF
:1031F000C046C046C046054908699A61000A033ABC
:10320000C0B29A617047C0460008004800040048F8
:1032100070B504000D000022AA210F48FFF7A4FF9B
:10322000002255210D48FFF79FFF0022A0210A48E8
:10323000FFF79AFF002229002000FFF795FF0021E9
:103240002000FFF7C1FF0500C04600212000FFF766
:10325000BBFF8542F3D170BDAA8A000055850000EE
:1032600070B504000D000022AA210F48FFF77CFF73
:10327000002255210D48FFF777FF0022A0210A48C0
:10328000FFF772FF002229002000FFF76DFF0021E9
:103290002000FFF799FF0500C04600212000FFF73E
:1032A00093FF8542F3D170BD55550000AA2A000056
:1032B0009023DB0530B51C68134D09022C401C60BF
:1032C000DA68124C2A40DA60114A506102229A628E
:1032D000104A00B215682C4314605469E4B22143CB
:1032E00051618021C9009961002801DA01209862AA
:1032F000C046C046996201219961491899611368D5
:1033000005490B40136030BDFFEFFFFF000055552E
:103310000008004800040048FFFFAAAAF7B50123EF
:103320000225294F01923A780091054393400421E8
:10333000A020264E2D049BB229433268C00100F024
:10334000FFFC040001283DD13B7809209C40054347
:103350007830A3B232682900FF3000F0F1FC04009D
:1033600001282FD13B7832689C402900A3B200206D
:1033700000F0E6FC0400012824D1009B180AFFF7A6
:10338000E3FE3B7832689C402900A3B200F0D8FCF1
:103390000400012816D16B461878FFF7D5FE2200ED
:1033A0003B7829009A4093B2326800F0C9FC01983A
:1033B000FFF7CAFE3B7832689C402900A3B200F0B8
:1033C000BFFC0400E0B2FEBDF0060020EC060020C9
:1033D000F7B501230225274F00903A780191054364
:1033E00093400421C020244E2D049BB2294332680F
:1033F000800100F0A5FC0400012838D109231D43F9
:103400003B78C0209C403268A3B22900400000F005
:1034100097FC040001282AD13B7832689C4029009F
:10342000A3B2002000F08CFC040001281FD1019BF6
:10343000180AFFF789FE3B7832689C402900A3B246
:1034400000F07EFC0400012811D16B461879FFF7CB
:103450007BFE22003B789A4093B2009A14430922E3
:10346000E1B209041143326800F06AFC0400A0B222
:10347000FEBDC046F0060020EC06002000238000C0
:1034800080B2834200D17047C046C04601339BB230
:10349000F7E700000F4B30B59022586180230124DC
:1034A000D205DB0093620C4B94621D680B48090245
:1034B000284318605869C0B201435961C0460821C9
:1034C0009162C04691611968054801401960946194
:1034D00030BDC046000800480004004800005555B3
:1034E000FFFFAAAA0B4B10B580215861902301223F
:1034F0000424DB05C90099619A629C62C046C046FB
:10350000C046054800699C61000A9962C0B29A6190
:1035100010BDC04600080048000400480E4B984209
:1035200002D880231B0218430C4B0D4A58610D4BE7
:103530000902186802431A605A69D2B211435961EC
:10354000C04690220821D2059162C04691611A6856
:1035500005490A401A607047FF1F00000008004834
:103560000000555500040048FFFFAAAA0A4B9842E4
:1035700002D880231B021843084B04225861902371
:10358000DB059A62C046C046C046C0460449086989
:103590009A61000AC0B27047FF1F0000000800488F
:1035A00000040048F8B505000E001C4F1C4B38887D
:1035B0002021203080B21C78FFF77AFEAA2119481A
:1035C000FFF7ACFF38881021103080B2FFF770FE93
:1035D00055211548FFF7A2FF38882021203080B2FE
:1035E000FFF766FEA0210F48FFF798FF24013888F7
:1035F000E4B2001980B22100FFF75AFE3100280022
:10360000FFF78CFF2800FFF7B1FF0400C046280039
:10361000FFF7ACFF8442F5D1F8BDC046340400206A
:103620008804002055150000AA0A000070B50400A7
:10363000B0200E0000020A21FFF73AFEC0200A2146
:103640000002FFF735FEAA211248FFF767FF552158
:103650001148FFF763FFA0210E48FFF75FFFB0207E
:103660000E4D00022978FFF723FEC02029780002C2
:10367000FFF71EFE31002000FFF750FF2000FFF78C
:1036800075FF0500C0462000FFF770FF8542F5D1A9
:1036900070BDC04655150000AA0A0000880400202D
:1036A00070B504000D000D48AA21FFF737FF552122
:1036B0000B48FFF733FFA0210848FFF72FFF290031
:1036C0002000FFF72BFF2000FFF750FF0500C0464A
:1036D0002000FFF74BFF8542F5D170BD5515000066
:1036E000AA1A000070B504000D001A4E022130889D
:1036F000023080B2FFF7DCFDAA211748FFF70EFF6A
:1037000030880121013080B2FFF7D2FD55211348E6
:10371000FFF704FF30880221023080B2FFF7C8FDB6
:10372000A0210D48FFF7FAFE0D4B3088197840189C
:1037300080B2FFF7BDFD29002000FFF7EFFE20005B
:10374000FFF714FF0500C0462000FFF70FFF85427A
:10375000F5D170BD3404002055150000AA0A000000
:103760008804002070B50400A0200D000002022192
:1037700000F0CEFAAA211048FFF7D0FE55210F48DD
:10378000FFF7CCFEA0210C48FFF7C8FEA0200C4B91
:103790000002197800F0BCFA29002000FFF7BEFEF5
:1037A0002000FFF7E3FE0500C0462000FFF7DEFE25
:1037B0008542F5D170BDC04655150000AA0A00002B
:1037C0008804002070B504000D000D48AA21FFF701
:1037D000A5FE55210B48FFF7A1FEA0210848FFF7E1
:1037E0009DFE29002000FFF799FE2000FFF7BEFE96
:1037F0000500C0462000FFF7B9FE8542F5D170BD37
:1038000055150000AA0A00000D4B80225861902334
:10381000D200DB0500B29A61002801DA01229A6227
:10382000C046C046C046C046064B80221869902359
:10383000D200DB059A620122000AC0B29A61704789
:10384000000800480004004870B504000D0010484E
:10385000AA21FFF72DFD55210E48FFF729FDA021D4
:103860000B48FFF725FD29002000FFF721FDA020D0
:10387000094B00021978FFF71BFD2000FFF7C4FF7A
:103880000500C0462000FFF7BFFF8542F5D170BD9F
:10389000AAFA000055F500008804002070B5040065
:1038A0000D001048AA21FFF703FD55210E48FFF730
:1038B000FFFCA0210B48FFF7FBFC29002000FFF7CD
:1038C000F7FC802000210002FFF7F2FC2000FFF748
:1038D0009BFF0500C0462000FFF796FF8542F5D10B
:1038E000280070BD55D50000AAAA000070B50400DC
:1038F0000D00134E00213088FFF7DAFCAA21114891
:10390000FEF712FD55211048FEF70EFDA0210D48CF
:10391000FEF70AFD0D4B30881978401880B2FFF78A
:10392000C7FC29002000FEF7FFFC2000FFF76CFF1A
:103930000500C0462000FFF767FF8542F5D170BD46
:103940003404002055550000AA2A000088040020F5
:1039500070B50400C0200D000002052100F0D8F968
:10396000AA210D48FFF7A4FC55210C48FFF7A0FC45
:10397000A0210948FFF79CFC29002000FFF798FCD4
:103980002000FFF741FF0500C0462000FFF73CFF85
:103990008542F5D170BDC04655550000AAAA000069
:1039A00070B504000D000D48AA21FEF7BDFC55219D
:1039B0000B48FEF7B9FCA0210848FEF7B5FC29002A
:1039C0002000FEF7B1FC2000FFF71EFF05002000DD
:1039D000FFF71AFF8542F6D1280070BD555500004B
:1039E000AA2A00000D4B0E4A58610E4B09021868B6
:1039F00002431A605A69D2B2114390225961802160
:103A0000D205106849010143116040219162916122
:103A10001A6805490A401A607047C0460008004805
:103A20000000555500040048FFFFAAAAF7B504009E
:103A30000E004D7AC046C046C046C046C046C0468D
:103A4000C046C046C0460022AA215848FFF78CFB5A
:103A5000002255215648FFF787FB2402002220212F
:103A60005248FFF781FB23B20193EBB20093337A04
:103A7000AB4217D26B4680201B78002273729021D4
:103A80000002FFF771FB0022802011000002FFF707
:103A90006BFB80200022F0210002FFF765FBC0468F
:103AA0000020FEBD434B444A196808200A43FF2109
:103AB0001A605A690A40A02109020A435A619022F9
:103AC0000121D20590629162C046C046C046C04600
:103AD000FF24906191611A6838492C400A401A60AD
:103AE000019B009A1C437368A4B2995C20000022D9
:103AF000FFF73AFBC046C046C046C046C046C04677
:103B0000C046C046C046C04600212000FFF75CFB0F
:103B10000700C046C046C046C046C046C046C04674
:103B2000C046C0467368009A9B5C834217D0C0466B
:103B3000C046C046C046C046C046C046C046C04655
:103B400000212000FFF740FBB8420BD1C046C04621
:103B5000C046C046C046C046C046C046C046013505
:103B6000ADB282E7C046C046C046C046C046C04669
:103B7000C046C046C046C046C046C046C046C04615
:103B8000C046C046C046C046C046C046C046C04605
:103B9000C046C046C046C046C046C046C046C046F5
:103BA00000212000FFF710FB0700C9E7AA8A0000E8
:103BB000558500000004004800005555FFFFAAAAE3
:103BC000F0B51C4D040005A8067868690902C0B26A
:103BD0000843686190200421C00581622900002A01
:103BE00001D101328262FF2500204A692D022A405C
:103BF0001A43114F4A61C046C046C046C046C0463F
:103C0000C046C046C046C046C0463A690133120AA3
:103C100022544A69DBB22A4001301A43C0B24A61D9
:103C2000B042E8D990230422DB059A61033A9A61F5
:103C3000F0BDC0460008004800040048F0B5184C2C
:103C4000050060690E02C0B230436061802690209A
:103C5000F600C00549B28661002901DA01218162BE
:103C6000FF2661693602314011436161C046002080
:103C70000C4FC04639690132090A29546169D2B230
:103C8000314001301143C0B261619842F1D99023B3
:103C90008022DB05D2009A6201229A61F0BDC04603
:103CA0000008004800040048F0B5174C05000E005D
:103CB00060691F2925D8802131430902C0B2014320
:103CC000616190210420FF26C9058862616936027E
:103CD000314011436161C04600200C4FC046396934
:103CE0000132090A29546169D2B2314001301143CD
:103CF000C0B261619842F1D990230422DB059A6138
:103D0000F0BDC0B20902DAE700080048000400482C
:103D100070B506000D0005243000013CFFF774FD6E
:103D2000E4B229003000FFF7C3FA6D08002CF3D18C
:103D300070BD00008047C046000000000000000089
:103D4000F0B5474680B4061C081C000C102801D5AD
:103D5000162700E004270007000F8046FF200140DF
:103D60005468251C1D439C43F60313850AD5C046A1
:103D7000C046C046C046C046C046C0469480138375
:103D8000958002E0012000F081F801390AD4381C46
:103D900000F07CF8C046948013839580C046C046EE
:103DA0007600E2E7381C013800F070F89480138345
:103DB0009580042000F06AF8108A184001D0FF2096
:103DC00061E0C046C046C046C046C046C04694807A
:103DD0009580108A184055D001200226B04552D057
:103DE0000921168A1E40FCD1012000F04FF8948072
:103DF000C0469580C04603E0C046C046C046C046A7
:103E0000948095807600108A1840EFF3008040007F
:103E1000C00F0643381C023800F038F894809580B3
:103E2000022000F033F80139EAD51385948001208F
:103E300000F02CF813839580301C802102239940D8
:103E40000E401BD1002341085E4149085E414908EC
:103E50005E4149085E4149085E4149085E414908A2
:103E60005E4149085E4149085E41760808D3400832
:103E7000FF21084048400002013004E00E2002E02B
:103E8000092000E0002080BCB846F0BD0138FDD11B
:103E90007047C04603685A0003D45B005B08C01833
:103EA0007047802212061343F9E7C046F0B5574623
:103EB0004E46DE464546E0B5814683B0924600292F
:103EC00025D04B1E9B46002701935B46FB18DC0F59
:103ED000E4184B466410E5005E193000FFF7DAFF86
:103EE000019B8046A3420BD0280008304844FFF7CE
:103EF000D1FFD04506D80138504509D2671CE4E708
:103F0000504505D9A74202D0631E9B46DDE7002637
:103F1000300003B03CBC90469946A246AB46F0BD8B
:103F2000012809D0022805D0002801D000207047C0
:103F30000248FCE70248FAE70248F8E74146000871
:103F4000594600084D46000830B5234B83B00500A4
:103F50008C1E002B2AD001A9200000E000BF002801
:103F600020D001992200FFF7A1FF041E1AD0FFF70D
:103F700091FF6368A864012B10D0201D002B1BDB70
:103F8000FFF788FF0023E8642B650368002B17DB2D
:103F9000FFF780FF2861002003B030BD002305201B
:103FA0002B61F9E7002309202B61F5E70B480C4949
:103FB000091AC9100191D5E70123E8642B65E4E7EC
:103FC0001801000FFFF7ACFF2861002801D109306C
:103FD000E2E70020E0E7C04600000000484F00088C
:103FE00018500008036810B50400DA0705D49B07D1
:103FF0000FD5483000F084FC23685A070FD51A0704
:1040000014D5DB0604D42000D130FF3000F084FC4E
:1040100010BD483000F070FC23685A07EFD4200030
:10402000D03000F071FC23681A07EAD42000513028
:10403000FF3000F06DFC2368E3E7C0460368002B07
:1040400000D01B1818007047092070477047C04601
:1040500070B504000D0008E02B6C2A00636121009C
:10406000012023699847082807D1296C2000FFF711
:104070006BFF0028F0D000F09FFE0728FBD1002046
:10408000296CFFF7E3FF281D00F020FCF0B5CE46B9
:10409000474680B5C368324C9846A54483690600FC
:1040A00014000431402205A8994600F08DFE00233B
:1040B00004AD296C30000493FFF746FF631E9C415A
:1040C00007000934002F15D0AB6B10216B644B46F1
:1040D00021430193C9B20095330032000120C0474B
:1040E000002833D13800F5239B009D440CBC90463A
:1040F0009946F0BDF0222B6C5200736129007CA818
:1041000000F062FE7CAA31003369200098478A9B48
:1041100007006B6403934B46009501933200330014
:1041200021000120C047002810D1F0227CA95200B4
:10413000280000F049FE082F06D1296C3000FFF757
:1041400003FF09240700BDE7072F01D00927C9E7AE
:104150000020296CFFF77AFF05A800F0B7FBC046E6
:104160002CFCFFFF406C704770B5CB6BFAB00B6452
:1041700004000E004022043103A800F025FE0123B4
:104180005B42029306E002AA2100236998470500DA
:1041900008280AD1129B200019000193FFF7D4FED2
:1041A0000028F0D009207AB070BD02A8FFF71AFFEE
:1041B000062DF7D131002000FFF74AFF10B58261CC
:1041C000DA6BC1601A6419000022FFF75FFF10BDAF
:1041D000436970B50B64C36804000D00002B04D064
:1041E0000122FFF753FF00F0E7FD0A0023690100F9
:1041F00002209847072807D0082803D1290020006B
:10420000FFF726FF00F0D8FD0020296CFFF71EFF06
:10421000281D00F05BFBC046C36810B5002B05D01D
:10422000CB6B00220B64FFF731FF10BDFFF79CFF43
:10423000FBE7C0467047C046836810B5002B02D02C
:1042400001000120984710BD10B5012907D00029B1
:1042500007D003390224012901D9200010BD01240F
:10426000FBE70224002BF8D10F2AF6D8920082181F
:104270005268029B00241A60EFE7C04600B585B083
:1042800003AB0A00009300210023FFF7DDFF039832
:1042900005B000BD10B5012907D0002907D00339AA
:1042A0000224012901D9200010BD0124FBE70224CA
:1042B000002BF8D10F2AF6D8029B92001B688218B7
:1042C00053600024EFE7C04600B585B003AB03920E
:1042D00000930A0000230021FFF7DCFF05B000BDBA
:1042E00070B51A4CD36BA544136406000D0019A8D1
:1042F000111D402200F068FD01235B42189314E079
:104300000C2118A802AAFFF7DFFF290018A8B04760
:10431000002812D1069B18AA02A9083001939847D9
:10432000040005280AD0092807D0289B02A81900F4
:104330000193FFF709FE0028E2D0092418A8FFF72F
:1043400051FE200090239B009D4470BDC0FDFFFFE7
:10435000F0B5DE464E464546574693460322E0B545
:104360001E0013008BB003400193CB6C0D001C1D8D
:104370001B6808940793002E66D11B02079306ABB7
:104380005E731A73019B022B00D16EE02B6DDB076D
:1043900047D40023A846B246029308330340039350
:1043A0002568002D00D137E15346022B49D02588DE
:1043B000668804340123370099469F4343469B6C2B
:1043C0000F219C4658466744FFF758FF002287425A
:1043D00006D82A004B469A43D719B8428041424238
:1043E00002230121760033400D402B43012B3ED0A8
:1043F000002B5AD0022B1CD1236801995F007F0843
:10440000002965D1002A06D0039A002A00D188E04D
:10441000002F00D1AAE0002B65DB0137BF00E419B3
:10442000BEE700230293022E47DDFFF70DFE0028B2
:1044300049D009200BB03CBC90469946A246AB46F9
:10444000F0BD66680834B5E7022E9BDC1A0C1B042D
:104450000793022306A90B73FD3313409B00E41856
:10446000019B4A73022B00D090E7AC6B8EE7019B57
:10447000002B3AD1002A16D02368DD0F63689A1CFE
:10448000D7D0424658320692013300D1C6E0201DF3
:10449000FFF7D4FD06AB01002A00404600E000BF54
:1044A000002800D0A7E008347AE7019B002B02D057
:1044B000002A00D08BE0043472E707A9584600F0C8
:1044C000D1FA0028B5D1029B002B5DD10820B1E7BD
:1044D00043460D2158461D6AFFF7D0FE854263D042
:1044E0002368002B99DA043497E743460D21584698
:1044F0001D6AFFF7C3FE8542D5D143469B6A9C42A5
:10450000D1D145462000FFF7C5FC0F2102005846D7
:10451000FFF7DAFE58462A000021FFF7D5FE0720F4
:1045200088E7002F22D058235146434406AABA46B2
:10453000251D0026049405911F00914603E00435D3
:104540002600A24514D028000697FFF777FD4B46BA
:10455000010000224046741C00E000BF0028EED09D
:104560005746059B049C9A46B742B9D1454601E09F
:104570004546049C0D215846FFF780FE069B2862A5
:104580006B62AC62062055E70F215846FFF776FEB6
:104590000E2102005846FFF797FE5846274A0F2182
:1045A000FFF792FE072045E743469B6A9C4297D15E
:1045B000434642469F620023D36204331363231DA4
:1045C00053632368002B32DB0123029325E720008D
:1045D000FFF760FC454604340600AC63404600E04B
:1045E00000BF002800D124E7584632000F21FFF712
:1045F0006BFE07201EE707000D2158464546FFF7D2
:104600003DFE2862022F0FD1069BEB6243462C33FE
:104610006B62AC6206200DE7564604E70D21584652
:104620004546FFF72BFE2862069B6B62F1E73800D8
:10463000013080004546201865E7C04600000000B4
:1046400010B50023FFF784FE10BDC04610B501234E
:10465000FFF77EFE10BDC04610B50223FFF778FEBF
:1046600010BDC046F0B5CE46474680B50600C3B083
:1046700014001D0001294ED0002933D003290AD08F
:10468000042902D1002B00D189E0022043B00CBCE8
:1046900090469946F0BD032BF7D11404150C240C59
:1046A0002B19102BF1D8082203681A4200D0E7E03A
:1046B00020AB1800984600F02DF9B36BED001A00FE
:1046C000002C09D0E400EA1A1C1942441968D150A0
:1046D00004339C42FAD12200B263404600F018F93C
:1046E0000020D3E70220002BD0D1002301271004A3
:1046F000B56B000C321D39009940084202D0296880
:104700000435116001330432102BF4D10020A304CE
:10471000BCD4B563BAE71404170C240C012B5FD08A
:10472000052BB2D13B19202BAFD80F2F7DD9A14635
:10473000002C65D1002223009146B16B002B00DCD8
:1047400088E020A88046FA00DB00521ACB184244C9
:104750000868505004318B42FAD119004B46002BA7
:1047600010D04B4658003A00102F00D210220023E0
:10477000103AD2006A448000CC58D45004338342AB
:10478000FAD1C918012D5ED0B1630F2F74D94B46F1
:10479000002BA5D0684600F0B7F8002076E7102A75
:1047A00000D972E7102203681A4245D120AB1800E5
:1047B000984600F0B3F800230120B16B02009A4044
:1047C000144204D045460F689A00AF5004310133BB
:1047D000042BF3D14046B16300F09EF8002055E76A
:1047E0003B19102B00D950E70F2F00D94DE70023BC
:1047F0009946012233681A4230D14B46002B5AD0D9
:10480000042233681A4242D1012D47D00F2F06D817
:1048100020AB180000F076F84B46002B8AD0684693
:1048200000F074F81023DB1B87E7102BDFD9102270
:10483000524291469944DCE793430360D130FF3004
:1048400000F06CF8B2E7043120A8B16300F054F82E
:1048500000201BE74B46002B84D193E719009143BE
:104860000A003160052D1ED00322300093433360CF
:10487000483000F043F8C0E720A800F041F886E790
:10488000934303605130FF3000F044F810E73000EC
:1048900093433360D03000F039F8B5E720AB18000F
:1048A00000F02CF8BEE7022330001A433260483093
:1048B00000F028F8A1E7012D03D00F2F00D939E728
:1048C000A6E720AB180000F019F833E7011C3431DB
:1048D00038C9043B9C461D60A646011C20313CC9DA
:1048E00090469946A246AB46011C0831FCC9416876
:1048F0000068E54600BDC0467047C0467047C046E8
:104900007047C0467047C0467047C0467047C046B3
:104910007047C0467047C0467047C0467047C046A3
:1049200001B401A801B585B0FFB408A841464A46C4
:1049300053465C4665463EC001A83EC80F980090AD
:1049400000230CB401A9FFF70FFC109B12B018470D
:1049500001B401A801B585B0FFB408A841464A4694
:1049600053465C4665463EC001A83EC80F9800907D
:1049700000230CB401A9FFF72BFC109B12B01847C1
:1049800001B401A801B585B0FFB408A841464A4664
:1049900053465C4665463EC001A83EC80F9800904D
:1049A00000230CB401A9FFF737FC109B12B0184785
:1049B00001B401A801B585B0FFB408A841464A4634
:1049C00053465C4665463EC001A83EC80F9800901D
:1049D00000230CB401ABFFF7F1FB109B12B018479A
:1049E00001B401A801B585B0FFB408A841464A4604
:1049F00053465C4665463EC001A83EC80F980090ED
:104A000000230CB401AAFFF76BFC109B12B01847EF
:104A1000027A0300002A04D1427AB020002A07D18A
:104A20007047013A02720268100E12021A60F7E72C
:104A3000013A5A725A68111D59600321126819729D
:104A4000F2E7C04600B585B003AB00930C2200230B
:104A50000021FFF7F9FB039805B000BD10B5FFF783
:104A6000F1FF10BDF0B557464E464546DE460023E1
:104A7000E0B587B003930F339846083B99468023EF
:104A80001B0306000F009A463800FFF7C1FF040021
:104A9000B02821D0030632D4FF2583001D4005AB8A
:104AA0009B4600930D220023002130000435FFF7C0
:104AB000CBFB63064CD5059B5D1B05955B460093C0
:104AC00000230D2200213000FFF7E4FB3800FFF740
:104AD0009FFF0400B028DDD1039B0024002B2FD1C1
:104AE00005AD00950E2200213000FFF7ADFB0095CB
:104AF00000230F2200213000FFF7CCFB20E0030051
:104B000042469343DBB2802B63D0902B25D0A02B61
:104B100032D0B02B45D0C02B00D173E003004A4601
:104B20009343DBB2D02B0AD15346024001321A43E1
:104B3000052301213000FFF795FD0028A4D00924AA
:104B4000200007B03CBC90469946A246AB46F0BD5B
:104B5000059B9C4665440595B0E7833B03400D2BC0
:104B6000EDD0424605AD0240009500230021300003
:104B7000FFF76AFB0095A3E7FF234A461B011900D4
:104B8000824311410A001A40030702D58023DB014A
:104B90001A43002300213000FFF764FD0028CED126
:104BA00072E7B1284AD0B2285ED0B32800D18BE09A
:104BB000FC230340B42BC2D04A4653460240013284
:104BC0001A43012101233000FFF74CFD0028B6D124
:104BD0005AE704023800FFF71BFF802520432D020F
:104BE000A842ACD004010005020C002300213000D3
:104BF000FFF738FD0028A2D12C4200D144E7012361
:104C0000039341E7C6286AD0C7287CD003004A46F0
:104C10009343DBB2C02B00D18BE0C82800D18FE0DA
:104C2000C92800D08BE73800FFF7F2FEF02302031B
:104C30001B03134042460240013278E73800FFF779
:104C4000E7FE002800D17AE7030042469343DBB237
:104C5000002B00D073E7020000213000FFF702FDB7
:104C6000002800D06BE70FE705AB00939B460D22B1
:104C7000002300213000FFF7E7FA3800FFF7C8FEF5
:104C800003066AD57F25B03C059B2840A0409C4682
:104C90006044059038000734FFF7BAFE0306F3D4EA
:104CA000812292009446863AFF3A1040A040059B2C
:104CB000723A634418185B46059000930021002364
:104CC0003000FFF7E7FADFE63800FFF7A1FEF02338
:104CD00002031B03134042460240013270E73800D2
:104CE000FFF796FEF02302031B03134042460240E7
:104CF00001321A43032303213000FFF7B3FC0028DD
:104D000000D01CE7C0E63800FFF782FE002800D183
:104D100015E7030042469343DBB2002B00D00EE7B9
:104D2000020004213000FFF79DFC002800D006E7B8
:104D3000AAE64346A0221C40013412032243D9E7CD
:104D40003800FFF765FE434602009A43D2B21032A4
:104D50001840120301300243EAE60224A0E7C046ED
:104D6000030000B5DB6C85B05A680800120201929E
:104D70001A0001A908324A6003220A72DB794B72D9
:104D8000FFF770FE05B000BD10B5FFF767FE806C41
:104D900010BDC04610B5FFF761FEC26CD3799B0011
:104DA0000833D01810BDC04610B500F005F8C04655
:104DB00010B5FFF7F9FFC04610B5062000F074F8F3
:104DC000012000F0A3F8C046F0B505000F2A2FD946
:104DD0000B0003439B0734D116000C000300103E68
:104DE000350901352D01451927681F6067685F6027
:104DF000A7689F60E7681034DF6010339D42F3D1ED
:104E00000F239E431036851989191340032B1AD995
:104E10001E1F0023B4080134A400CF58EF50043300
:104E2000A342FAD10324A643331D2240C918ED182A
:104E3000002A05D00023CC5CEC5401339342FAD114
:104E4000F0BD0500F6E71A00F2E7C04670B50500B0
:104E50000C001F2922D8B7239B00C358002B14D065
:104E60008A009B181A68002A0FD0012A0BD0511C07
:104E700005D00021200019609047002070BD162346
:104E800003600120FAE70020F8E7280000F02AF884
:104E900022000100280000F011F8EFE7162303605C
:104EA00001204042EAE7C04610B5034B01001868F4
:104EB000FFF7CCFF10BDC04600000020002370B5F6
:104EC000074C050008001100236000F017F8431C90
:104ED00000D070BD2368002BFBD02B60F9E7C046E3
:104EE0002407002010B500F001F810BD5822012061
:104EF000014B40421A6070472407002058220120CD
:104F0000014B40421A60704724070020FEE7C0466C
:084F1000F8B5C046F8B5C04633
:104F180074B20181B0AB308000000000800A0181CA
:104F2800B0B0ABF0000000003F020181B0AB3080B0
:104F38000000000080060181B0B0ABF00000000066
:104F4800ECEDFF7FB0B0B08044EFFF7F01000000C0
:104F5800F0EFFF7FB0A9028084F0FF7FB0B0A88097
:104F6800D4F0FF7F01000000E0F0FF7FB0B0AA801E
:104F780014F1FF7F9CFFFF7FE4F1FF7F0100000039
:104F8800E0F1FF7FAA3F39802CF2FF7FB0B0A88004
:104F980038F2FF7FB0B0AA8078F2FF7FB0B0A88067
:104FA8008CF2FF7F0100000088F2FF7FB0B0A8807C
:104FB80090F2FF7F0100000020F3FF7FAA0FB2806C
:104FC80088F3FF7F58FFFF7F70F6FF7FB0B0A8809F
:104FD8008CF6FF7F54FFFF7FECF8FF7F0100000095
:104FE8005CFAFF7F008404806CFAFF7FB0B0A88071
:104FF8006CFAFF7F40FFFF7F60FDFF7F0084048025
:1050080080FDFF7FB0B0A88098FDFF7F0100000001
:10501800080000200000000000000000F40200204A
:105028005C030020C4030020000000000000000012
:105038000000000000000000000000000000000068
:105048000000000000000000000000000000000058
:105058000000000000000000000000000000000048
:105068000000000000000000000000000000000038
:105078000000000000000000000000000000000028
:105088000000000000000000000000000000000018
:105098000000000000000000000000000000000008
:1050A80000000000000000000000000000000000F8
:1050B80000000000000000000000000000000000E8
:1050C80001000000000000000E33CDAB34126DE685
:1050D800ECDE05000B0000000000000000000000EE
:1050E80000000000000000000000000000000000B8
:1050F80000000000000000000000000000000000A8
:105108000000000000000000000000000000000097
:105118000000000000000000000000000000000087
:0400000508000801E6
:00000001FF
